:020000040800F2
:1000000000000220816200085D6100085F61000855
:10001000616100086361000865610008000000007C
:100020000000000000000000000000006761000800
:1000300069610008000000006B6100086D61000844
:10004000D5620008D5620008D5620008D5620008B4
:10005000D5620008D5620008D5620008D5620008A4
:10006000D5620008D5620008D562000875610008F5
:10007000D5620008D5620008D5620008D562000884
:10008000D5620008D562000885610008D5620008C5
:10009000D5620008D5620008D5620008D562000864
:1000A000D5620008D5620008D5620008D562000854
:1000B000D5620008D5620008D5620008D562000844
:1000C000D5620008D5620008D5620008D562000834
:1000D000D5620008D5620008D5620008D562000824
:1000E000D5620008D5620008D5620008D562000814
:1000F000D5620008D5620008D5620008D562000804
:10010000D5620008D5620008D5620008D5620008F3
:10011000D5620008D5620008D5620008D5620008E3
:10012000D5620008D5620008D5620008D5620008D3
:10013000D56200080000000000000000D562000841
:10014000D5620008D5620008D5620008D5620008B3
:10015000D5620008D5620008D5620008D5620008A3
:10016000D5620008D5620008D5620008D562000893
:10017000D5620008D5620008D562000800000000C2
:10018000D5620008D5620008D5620008D562000873
:10019000D5620008D5620008D5620008D562000863
:1001A000D5620008D5620008D5620008D562000853
:1001B000D5620008D5620008D5620008D562000843
:1001C000D5620008D56200080000000000000000B1
:1001D0000000000000000000D562000800000000E0
:1001E000000000000000000000000000000000000F
:1001F0000000000000000000D5620008D562000881
:10020000D5620008D562000800000000D562000831
:10021000D5620008D5620008D5620008D5620008E2
:10022000D5620008D5620008D56200080000000011
:10023000D5620008D562000800000000D562000801
:10024000D5620008D5620008D5620008D5620008B2
:10025000D5620008D5620008D5620008D5620008A2
:10026000D5620008D5620008D5620008D562000892
:10027000D5620008D5620008D562000800000000C1
:10028000D5620008D562000800000000D5620008B1
:1002900000000000D5620008D562000800000000E0
:0C02A00000000000D5620008D5620008D4
:1002AC0010B5054C237833B9044B13B10448AFF3A4
:1002BC0000800123237010BD1000002000000000FE
:1002CC004C63000808B5034B1BB103490348AFF35B
:1002DC00008008BD00000000140000204C630008E2
:1002EC0030B585B00024009401940294039401F07D
:1002FC0077FA01238DF800308DF8014001941F220C
:10030C008DF8082087228DF809208DF80A408DF889
:10031C000B408DF80C308DF80D308DF80E408DF8AB
:10032C000F40684601F07AFA042001F067FA05B034
:10033C0030BD00002DE9F0418AB005AD00240594D4
:10034C000694079408940994434BD3F8402142F047
:10035C008002C3F84021D3F8402102F080020092C1
:10036C00009AD3F8402142F00402C3F84021D3F89C
:10037C00402102F004020192019AD3F8402142F08C
:10038C000102C3F84021D3F8402102F0010202928D
:10039C00029AD3F8402142F00202C3F84021D3F86C
:1003AC00402102F002020392039AD3F8402142F05A
:1003BC000802C3F84021D3F8403103F0080304933A
:1003CC00049B264E22464CF20441304602F070FC4F
:1003DC00234F22464FF48051384602F069FC4CF210
:1003EC00044305934FF00108CDF818800794089446
:1003FC002946304602F04CFB4FF480530593CDF860
:10040C001880079408942946384602F041FB4FF4B3
:10041C0000430593069407942946384602F038FBAE
:10042C004FF4E05305930694079429460D4802F0C7
:10043C002FFB042305930694079429460A4802F0DF
:10044C0027FB10230593069407942946304602F0A7
:10045C001FFB0AB0BDE8F0810044025800040258AA
:10046C000000025800080258000C025800B583B076
:10047C000B4BD3F8382142F00102C3F83821D3F8E2
:10048C00383103F001030193019B002211460B202C
:10049C0001F07EF90B2001F08BF903B05DF804FB41
:1004AC000044025872B6FEE700B58BB000230793E8
:1004BC000893099300930193029303930493059378
:1004CC0006932048204A026043608360C360082280
:1004DC000261037543750122826103774FF4B462A4
:1004EC0042624FF480628262C3624FF480520263B4
:1004FC00436380F8383000F071FFE8B900230793AC
:10050C0007A9104801F06CF8C0B9104B00930623F2
:10051C0001930323029340F2FF7303930423049388
:10052C00002305938DF819306946064800F0C6FC87
:10053C0030B90BB05DF804FBFFF7B4FFFFF7B2FF67
:10054C00FFF7B0FF60030020002002400800900C71
:10055C0008B51548154B036000238360C360037412
:10056C004374837403224261012282610D21C161B3
:10057C000221016242628262C2620263436383634C
:10058C00C3630364042242648364C26403654265EA
:10059C008365C36503664366826602F02FF900B972
:1005AC0008BDFFF77FFF00BF4802002000A00040FD
:1005BC0008B51548154B036000238360C3600374B2
:1005CC004374837403224261012282610D21C16153
:1005DC000221016242628262C262026343638363EC
:1005EC00C3630364042242648364C264036542658A
:1005FC008365C36503664366826602F0FFF800B943
:10060C0008BDFFF74FFF00BFA801002000A4004069
:10061C0010B59CB00024189419941A941B9415943A
:10062C00169417940E940F9410941194129413948E
:10063C0014943422214601A805F047FE3A483B4B5E
:10064C000360446084604FF6FF73C36004614461CF
:10065C00846105F00BFA002853D14FF480531893A2
:10066C0018A9314805F038FC00284CD12E4805F06B
:10067C002DFA002849D1002315931693179315A929
:10068C00294805F0C5FC002841D160230E930022B7
:10069C000F92109211921292139214920EA9224858
:1006AC0005F0BEFA002834D104220EA91E4805F02C
:1006BC00B7FA00282FD108220EA91B4805F0B0FA72
:1006CC0058BB0C220EA9184805F0AAFA38BB002317
:1006DC00019302930393049305934FF400520692F3
:1006EC00079309934FF000720A920B930D9301A993
:1006FC000D4805F0DDFCA0B90B4802F0C7FC1CB09E
:10070C0010BDFFF7CFFEFFF7CDFEFFF7CBFEFFF7D7
:10071C00C9FEFFF7C7FEFFF7C5FEFFF7C3FEFFF7E5
:10072C00C1FEFFF7BFFE00BF5C01002000000140CE
:10073C0000B58BB0002307930893099300930193A2
:10074C00029303930493059306931A481A4A026082
:10075C00436083604FF6FF72C2600361836105F0F2
:10076C00B5F9F8B900230793099307A9114805F0C7
:10077C004FFCC8B9602300930023019302930493A8
:10078C00042269460B4805F04BFA78B90C226946ED
:10079C00084805F045FA58B9064802F077FC0BB04A
:1007AC005DF804FBFFF77EFEFFF77CFEFFF77AFE99
:1007BC00FFF778FE100100200004004000B58BB05C
:1007CC0000230793089309930093019302930393D7
:1007DC000493059306931A481A4A02604360836097
:1007EC004FF6FF72C2600361836105F06FF9F0B9D7
:1007FC0000230793099307A9114805F009FCC0B918
:10080C0060230093002201920292049269460C48E4
:10081C0005F006FA78B904226946094805F000FA91
:10082C0058B9074802F032FC0BB05DF804FBFFF737
:10083C0039FEFFF737FEFFF735FEFFF733FE00BF3B
:10084C00C40000200008004000B589B000230593C7
:10085C0006930793019302930393049319481A4A3E
:10086C000260436083604FF6FF72C26003614361B4
:10087C00836105F05BF9E8B90023059306930793B0
:10088C0005A9104805F0C4FBB0B900220192012360
:10089C0002930392049201A90A4805F0A9FA68B9D7
:1008AC0004220DEB0201074805F0A2FA40B909B089
:1008BC005DF804FBFFF7F6FDFFF7F4FDFFF7F2FD23
:1008CC00FFF7F0FD2C0000200004014000B585B0BE
:1008DC0000230193029303930D480E4A02600222F7
:1008EC00426083604BF68032C260836105F0BEF8D3
:1008FC0050B900230193039301A9054805F088FB27
:10090C0020B905B05DF804FBFFF7CCFDFFF7CAFD7D
:10091C00780000200010004000B59DB04C22002152
:10092C0009A805F0D2FC2022002101A805F0CDFC7D
:10093C00254B4FF0FF32C3F8B020022002F028FC08
:10094C0000230093214A936923F4404343F400436A
:10095C009361936903F440430093009B1B4B9B6989
:10096C0013F4005FFAD0012309934FF480330A93F8
:10097C00022312931393149320221592169303229D
:10098C00179218930C23199300231A931B9309A8FD
:10099C0002F028FC98B93F23019303230293002310
:1009AC00039308220492059306930793089302215C
:1009BC0001A803F043F820B91DB05DF804FBFFF764
:1009CC0071FDFFF76FFD00BF00440258004802584C
:1009DC0008B5FFF785FC00F081F8FFF79DFFFFF7E6
:1009EC00A9FCFFF743FDFFF75FFDFFF7B1FDFFF734
:1009FC00DFFDFFF70DFEFFF79BFEFFF7DFFEFFF7B6
:100A0C0023FFFFF763FF204C01224FF48041204667
:100A1C0002F04EF94FF4FA7000F0A0F800224FF4F7
:100A2C008041204602F044F94FF4FA7000F096F839
:100A3C0001224FF40041204602F03AF94FF4FA70CB
:100A4C0000F08CF800224FF40041204602F030F9FF
:100A5C004FF4FA7000F082F8A4F5806401224FF490
:100A6C008051204602F024F94FF4FA7000F076F829
:100A7C0000224FF48051204602F01AF94FF4FA701C
:100A8C0000F06CF8BFE700BF00040258104B1B7855
:100A9C000BB90120704710B504464FF47A70B0FBC7
:100AAC00F3F30C4A1068B0FBF3F000F085FE68B964
:100ABC000F2C01D901200AE0002221464FF0FF3013
:100ACC0000F066FE044B1C60002000E0012010BD0D
:100ADC00000000200C0000200400002010B50320B2
:100AEC0000F044FE02F0AEFE0F498B69C3F3032302
:100AFC000E4AD35C03F01F03D8408B6903F00F033D
:100B0C00D35C03F01F0320FA03F3094A1360094B6B
:100B1C0018600F20FFF7BAFF10B10124204610BD5A
:100B2C00044602F0CBF8F9E700440258B863000819
:100B3C00080000200C000020034B1B78034A1168AE
:100B4C000B441360704700BF00000020C40300205A
:100B5C00014B1868704700BFC403002038B5044629
:100B6C00FFF7F6FF0546B4F1FF3F02D0044B1B78AC
:100B7C001C44FFF7EDFF401BA042FAD338BD00BF69
:100B8C000000002010B430300B0A9B0003F00C0363
:100B9C00C45801F01F014FF01F0C0CFA01FC24EAA1
:100BAC000C0CC2F384628A404CEA0202C2505DF81B
:100BBC00044B704710B414304B0E9B0003F004032D
:100BCC00C458C1F304514FF0070C0CFA01FC24EA91
:100BDC000C0C8A404CEA0202C2505DF8044B704780
:100BEC00C1F313033BB9C1F3846101228A40C36989
:100BFC001343C361704791FAA1F131B1B1FA81F19C
:100C0C0001F01F0101228A40F1E72021F8E770472B
:100C1C0070477047F8B5044603681F685D689A4BC7
:100C2C009E6806F01F0617F0020F10D015F0020F89
:100C3C000DD0436D13F0100F03D1436D43F40063DB
:100C4C004365204600F0CAFC236802221A6017F0A4
:100C5C00040F02D015F0040F05D117F0080F4DD07A
:100C6C0015F0080F4AD0636D13F0100F03D1636DAC
:100C7C0043F4007363652368DA6812F4406F37D16C
:100C8C00824A934227D01A46934207D0092E25D880
:100C9C0040F22121F14011F0010F1FD0DA6812F45B
:100CAC00005F25D11A6812F0080F21D09A6812F053
:100CBC00040F15D15A6822F00C025A60636D23F4AC
:100CCC0080736365636D13F4805F11D1636D43F0C2
:100CDC00010363650CE0A2F58072D5E7D268DEE70C
:100CEC00636D43F010036365A36D43F00103A365CB
:100CFC002046FFF78CFF23680C221A6017F0200F98
:100D0C0002D015F0200F05D117F0400F63D015F06D
:100D1C00400F60D0636D13F0100F03D1636D43F47B
:100D2C00005363652368DA6C12F4C07F19D101217A
:100D3C00DA6812F4406F16D10120544A934214D051
:100D4C001A46934214D0062E14BF4FF0000C4FF0ED
:100D5C00010C6EB1BCF1000F0AD1072E08D0D2687D
:100D6C0007E00021E4E70020E7E7A2F58072E8E75E
:100D7C00DA6851B312F0007F03D030B312F4005F85
:100D8C0023D1196811F0400F1FD012F4001F1CD191
:100D9C009A6812F0080F10D15A6822F060025A605B
:100DAC00636D23F480536365636D13F4807F0CD102
:100DBC00636D43F00103636507E0636D43F010035B
:100DCC006365A36D43F00103A365204600F002FCAC
:100DDC00236860221A6017F0800F02D015F0800F84
:100DEC002FD117F4807F02D015F4807F34D117F403
:100DFC00007F02D015F4007F3AD117F0100F19D0F4
:100E0C0015F0100F16D0236B33B1002E40D01E4BB3
:100E1C009B6813F4404F0AD0636D43F480636365A1
:100E2C00A36D43F00203A3652046FFF7F2FE23688F
:100E3C0010221A6017F4806F02D015F4806F2DD138
:100E4C00F8BD636D43F4803363652046FFF7E0FE25
:100E5C00236880221A60C4E7636D43F40033636532
:100E6C00204600F0B9FB23684FF480721A60BEE78D
:100E7C00636D43F480236365204600F0AEFB23686A
:100E8C004FF400721A60B8E70023024000210240C0
:100E9C002368DB6813F0030FC9D0BDE7636D43F41F
:100EAC0080436365A36D43F00803A36523684FF487
:100EBC0080621A60204600F08EFBC1E7F0B583B06B
:100ECC000023019390F85030012B00F0FD81044673
:100EDC000D46012380F850300268936813F0040F1C
:100EEC0009D0436D43F0200343650120002384F8AF
:100EFC00503003B0F0BD0B68002B0ADBC3F31301B9
:100F0C0000293AD1C3F3846301219940D3690B437F
:100F1C00D3612A6869682068FFF734FE2068866808
:100F2C0016F0040600D00126836813F0080F00D1D8
:100F3C007EB32068816811F0010140F0C1812B68FB
:100F4C00EE68D0F8C020C3F3130C22EA0C0206F0B2
:100F5C00180C9B4E26FA0CF63340C3F313031343C1
:100F6C00C0F8C030EA68974B9A4200F08F802B682B
:100F7C00002BC0F206810020B8E793FAA3F333B13B
:100F8C00B3FA83F303F01F0301219940BEE720233A
:100F9C00F8E7AA682968FFF70DFE2368DA6812F0F3
:100FAC00100F31D16A69D968C1F3820149008A40B6
:100FBC002F69042F36D02868603353F8271001F0BE
:100FCC00004100F0F84002430A4343F8272023680D
:100FDC0028696A7E012A1FD03246603353F82010EC
:100FEC0021F000410A4343F82020206829692B7E18
:100FFC00012B14D0026922F4F04201F01F0306FA0F
:10100C0003F31343036194E76A69D968890801F013
:10101C00040149008A40CBE74FF00042DDE74FF472
:10102C000066E7E71A6E02F0F8422968B2EB816FAE
:10103C001DD02268536E03F0F8432968B3EB816F1F
:10104C001AD02268936E03F0F8432968B3EB816FD2
:10105C0017D02268D36E03F0F8432968B3EB816F85
:10106C007FF467AFD36E23F00043D36661E71A6E4B
:10107C0022F000421A66DCE7536E23F000435366FD
:10108C00DFE7936E23F000439366E2E720684E4B54
:10109C00984205D04D4B98422BD0FFF7A1FD66E747
:1010AC002B684B4A93424AD04A4A934249D04A4A07
:1010BC00934248D0494A934247D002F1866210329B
:1010CC00934244D0464A934243D002F1042202F5A3
:1010DC00401293423FD002F1866202F500629342C5
:1010EC003BD0404A93423AD03F4A9342D5D13F49F4
:1010FC00D3E72B68364A934233D0364A934232D0E8
:10110C00354A934231D0354A934230D002F186624F
:10111C00103293422DD0324A93422CD002F1042249
:10112C0002F54012934228D002F1866202F5006269
:10113C00934224D02C4A9342AFD12C49ADE70121E4
:10114C00ABE72B49A9E72B49A7E72B49A5E72B4987
:10115C00A3E72B49A1E72B499FE72B499DE72B4997
:10116C009BE7012199E7224997E7224995E7224914
:10117C0093E7224991E722498FE722498DE72249DB
:10118C008BE7234A916801F0E075A2F540729268F2
:10119C0012F0010200D001220C48806810F0010FFF
:1011AC0040F08880002A40F085801A4A934237D05C
:1011BC00194A934258D0194A934268D0002095E6B8
:1011CC00FFFF0F000000FF470020024000210240FB
:1011DC0002003004040060080800900C1000C010DD
:1011EC000004002A000021430000844B0000B84F8B
:1011FC00400020198000501D000180210002B02504
:10120C000008302E0010603200209036000052474B
:10121C0000230240000084CB0040C0BA0000B8CFCD
:10122C0011F4000FC4D12268284B9A4201D000203F
:10123C005CE645F4000326498A6822F0E072134309
:10124C008B60244B1B689B09234AA2FB03239B093D
:10125C0001335B00019302E0019B013B0193019B75
:10126C00002BF9D1002041E611F0807FA3D1226838
:10127C00164B9A4201D0002038E645F08073144991
:10128C008A6822F0E07213438B6000202EE611F482
:10129C00800F17D122680D4B9A4201D0002025E611
:1012AC0045F480030A498A6822F0E07213438B608C
:1012BC0000201BE6636D43F020036365012015E6F7
:1012CC00002013E6002011E6022012E60021024065
:1012DC00002302400C000020632D3E0510B504468F
:1012EC003A4B9B6813F4403F19D002F0F1FC636851
:1012FC00B3F5003F05D0B3F5403F0ED0B3F5803FBA
:10130C0002D11B0CB0FBF3F0314B984241D8226850
:10131C00936823F44073936010BD8008F4E74FF496
:10132C000020002103F04CFE6368B3F5101F2CD095
:10133C0021D8B3F5E01F26D004D9B3F5001FE3D1B3
:10134C004009E1E7B3F5801F10D009D8B3F5002FA1
:10135C000CD0B3F5402F09D0B3F5802F06D0D3E7CE
:10136C00B3F5A01F02D0B3F5C01FCDD19B0C5B0011
:10137C00B0FBF3F0C8E7B3F5201F08D0B3F5301F6E
:10138C00C2D1000AC0E70009BEE78009BCE7C0096A
:10139C00BAE7104B984207D82268936823F440733D
:1013AC0043F480739360B7E70B4B984207D82268DD
:1013BC00936823F4407343F400739360ACE72268A2
:1013CC00936843F440739360A6E700BF0023024088
:1013DC0021BCBE0041787D0181F0FA0230B583B0AA
:1013EC0000230193002800F0DF800446436DEBB12D
:1013FC0023689A6812F0005F03D099686B4A0A4020
:10140C009A6023689A6812F0805F1CD19968684AC8
:10141C000A4042F080529A60664B1B689B09664AF0
:10142C00A2FB03239B090133019309E001F058FC53
:10143C000023A36584F85030DAE7019B013B01934C
:10144C00019B002BF9D12268936813F0805F40F068
:10145C008180636D43F010036365A36D43F001035A
:10146C00A3650125936813F0040300D00123616D7B
:10147C0011F0100F40F09080002B40F08D80636DC8
:10148C0023F4817343F002036365936813F0010F37
:10149C0012D14A4B9B6813F0010300D00123484A38
:1014AC00926812F0010F07D133B9636845498A6815
:1014BC0022F47C1213438B60627D236B43EA42332C
:1014CC00A2681343227F43EA0243012A44D0626A92
:1014DC0022B102F47872A16A0A4313432168C868E6
:1014EC00394A02401A43CA602268936813F0040315
:1014FC0000D00123916811F0080F1CD1DBB9217DBC
:10150C00E36A43EA8131D068304B03400B43D3602C
:10151C0094F83830012B24D02268136923F001038E
:10152C0013612268136923F07043616B0B431361E1
:10153C002046FFF7D3FEE368012B24D02268136BFF
:10154C0023F00F031363636D23F0030343F00103D4
:10155C00636526E0002585E7226A013A43EA4243A7
:10156C00B5E7206802691A4B1340E26B511E226CDE
:10157C0042EA0142616C0A43A16C0A43134343F0F3
:10158C0001030361CDE721680B6B23F00F03A26904
:10159C00013A13430B63D6E7636D43F010036365A5
:1015AC000125284603B030BD0125FAE7C0FFFF5FD7
:1015BC00C0FFFF6F0C000020632D3E050020024091
:1015CC00002102400023024003C0F0FFFCBFFFFFDC
:1015DC001EF800FC7047704770477047704700005A
:1015EC0090F85020012A78D010B49BB00346012209
:1015FC0080F850200022169217920068384A9042C8
:10160C0031D000220192019A002A30D0926812F057
:10161C00040200D00122806810F0040F49D1002A86
:10162C0047D10A6862B32F48826822F440424C6862
:10163C00224382602A4A926812F0010200D00122F1
:10164C002948806810F0010F3FD1002A3FD1254C6A
:10165C00A068A2F5726202400868896801430A43D7
:10166C00A26000202AE002F580720192CBE75A6D4D
:10167C0042F020025A65002283F85020012020E01D
:10168C0018498A6822F440428A60154A926812F01E
:10169C00010200D001221449896811F0010F18D100
:1016AC00CAB910498868A2F5726202408A600020AB
:1016BC0004E05A6D42F020025A650120002283F8A2
:1016CC0050201BB05DF8044B70470020F6E700205B
:1016DC00F4E70020F2E70020F0E70220704700BF9B
:1016EC00002002400023024000210240002807DBBA
:1016FC0000F01F02400901239340024A42F82030B7
:10170C00704700BF00E100E0002804DB0901C9B20A
:10171C00044B1954704700F00F000901C9B2024B79
:10172C001954704700E400E014ED00E000B500F03F
:10173C000700C0F1070CBCF1040F28BF4FF0040CDC
:10174C00031D062B0FD9C31E4FF0FF3E0EFA0CF0F3
:10175C0021EA000199400EFA03FE22EA0E0241EA48
:10176C0002005DF804FB0023EEE700000649CB689D
:10177C0023F4E0631B041B0C000200F4E060034341
:10178C00024A1A43CA60704700ED00E00000FA05F7
:10179C0010B50446054BD868C0F30220FFF7C6FF0E
:1017AC0001462046FFF7B0FF10BD00BF00ED00E082
:1017BC0008B5FFF79BFF08BD0138B0F1807F0BD255
:1017CC004FF0E0235861054AF02182F823100020E5
:1017DC00986107221A6170470120704700ED00E004
:1017EC00BFF35F8F044B5A6A22F480325A62002294
:1017FC00C3F89420704700BF00ED00E040F00100FA
:10180C00054BC3F894005A6A42F480325A62BFF313
:10181C004F8FBFF36F8F704700ED00E04378144A91
:10182C00C2F89830D2F8A03023F00103C2F8A030EF
:10183C004368C2F89C30017BC37A1B0643EA0173F0
:10184C00817A43EAC143417B43EA8143817B43EA8A
:10185C004143C17B43EA0143417A43EA0123017AC4
:10186C0043EA410301780B43C2F8A030704700BF34
:10187C0000ED00E003682749274A934218BF8B42CA
:10188C002FD0183293422CD01832934229D01832D0
:10189C00934226D01832934223D01832934220D050
:1018AC00183293421DD002F55672934219D0183259
:1018BC00934216D01832934213D01832934210D060
:1018CC00183293420DD0183293420AD018329342F8
:1018DC0007D01832934204D023F0FF038365806D48
:1018EC00704710B4D9B210390C4AA2FB0142C2F3B2
:1018FC0002120B4CA25CC2655F2907D96FF3090376
:10190C0004338365806D5DF8044B70476FF30903F6
:10191C008365F7E71000024028000240ABAAAAAA90
:10192C00B063000883699BB9836A012B0AD0022B30
:10193C0002D00BB100207047C36A13F0807F2AD10C
:10194C0000207047C36AB3F1C07F26D000207047D7
:10195C00B3F5005F0AD0836A022B26D9032B26D15C
:10196C00C36A13F0807F24D100207047836A032B55
:10197C0003D8DFE803F01404140A00207047C36A8C
:10198C0013F0807F0DD100207047C36AB3F1C07F84
:10199C0009D00020704701207047012070470120BA
:1019AC0070470120704701207047012070470020CC
:1019BC00704701207047000003682149214A934277
:1019CC0018BF8B4227D01432934224D01432934246
:1019DC0021D0143293421ED0143293421BD01432B5
:1019EC00934218D01432934215D0DAB2103A1649F9
:1019FC00A1FB0212120915491944A8291ED9144B2E
:101A0C0013449B000366134B436602F01F02012331
:101A1C00934083667047DBB2083B0F4AA2FB03235B
:101A2C000E4A02EB1312920002660D4A4266C3F391
:101A3C000413012202FA03F3836670470832DEE7CF
:101A4C00085402581C540258ABAAAAAAF0FBFDBFBA
:101A5C000082001080080240CDCCCCCC0096001641
:101A6C008058025801794A1E072A2BD830B40368D3
:101A7C00154D164CA34218BFAB4218D01434A342D8
:101A8C0015D01434A34212D01434A3420FD0143402
:101A9C00A3420CD01434A34209D01434A34206D070
:101AAC000B4B0B449B00C3660A4B036705E00A4BC8
:101ABC000B449B00C366094B0367012393404367A8
:101ACC0030BC7047704700BF085402581C54025871
:101ADC003F820010400902403F96001640590258C0
:101AEC0070B50446FFF734F8002C00F0D981054698
:101AFC0023686349634A934218BF8B420CBF012190
:101B0C00002170D0183293426DD0183293426AD0B3
:101B1C001832934267D01832934264D018329342F1
:101B2C0061D0183293425ED002F5567293425AD06D
:101B3C001832934257D01832934254D018329342F1
:101B4C0051D0183293424ED0183293424BD01832A7
:101B5C00934248D01832934245D04B494B4A93425A
:101B6C0018BF8B4200F05481494A934200F05081D7
:101B7C001432934200F04C811432934200F04881AD
:101B8C001432934200F044811432934200F04081AD
:101B9C001432934200F03C813E4A934200F038816B
:101BAC001432934200F034811432934200F03081AD
:101BBC001432934200F02C811432934200F02881AD
:101BCC001432934200F024811432934200F02081AD
:101BDC001432934200F01C8140236365032384F884
:101BEC00353001204AE0022284F83520002284F8A6
:101BFC00342079BB284A93422CD01832934229D0F6
:101C0C001832934226D01832934223D01832934282
:101C1C0020D0183293421DD002F55672934219D03F
:101C2C001832934216D01832934213D01832934282
:101C3C0010D0183293420DD0183293420AD0183279
:101C4C00934207D01832934204D01A6822F0010252
:101C5C001A6003E01A6822F001021A6023681A68FD
:101C6C0012F0010F1AD0FEF773FF431B052BF5D9A9
:101C7C0020236365032384F83530012070BD00BF39
:101C8C001000024028000240082C02481C2C02487C
:101C9C00302C024808540258400002401A6881490E
:101CAC001140A268E0680243206902436069024364
:101CBC00A0690243E0690243206A02430A43616A55
:101CCC00042900F090806168522900F296803F2927
:101CDC00C0F08E803F39744820FA01F111F0010FE9
:101CEC0001D042F480121A602668756925F0070548
:101CFC00636A1D43042B08D1A36A1D43E36A23B115
:101D0C002046FFF70FFE00287CD175612046FFF7B7
:101D1C00B1FDE36D03F01F023F2393408360236802
:101D2C006249634A934218BF8B4242D018329342A5
:101D3C003FD0183293423CD01832934239D01832EB
:101D4C00934236D01832934233D01832934230D06B
:101D5C0002F5567293422CD01832934229D0183285
:101D6C00934226D01832934223D01832934220D07B
:101D7C00183293421DD0183293421AD01832934223
:101D8C0017D04C4A934214D01432934211D01432CF
:101D9C0093420ED0143293420BD01432934208D09B
:101DAC001432934205D01432934202D0143293422F
:101DBC0013D12046FFF700FEA368802B63D0236E5F
:101DCC0022791A60636EA26E5A606368013B072B1E
:101DDC005CD90023E36623676367002060650123F9
:101DEC0084F835304AE7E16A206B01430A436AE71D
:101DFC00293905293FF677AF73E7743903293FF684
:101E0C0072AF6EE740236365012084F8350035E737
:101E1C00022284F83520002284F8342019686FF3EC
:101E2C001011A268402A2CD0802A27D00022E0680A
:101E3C0042EAD002206942EAD002606942EAD0024A
:101E4C00A06942EAD002E06942EAD002206A42EA82
:101E5C0010120A431A602268174B1344174AA2FB4C
:101E6C0003231B099B00E3652046FFF703FDE26D8E
:101E7C0002F01F0101228A40426050E74FF4804279
:101E8C00D5E71022D3E70023636098E72046FFF7DD
:101E9C00E9FDE36E00221A60236F626F5A609CE7C3
:101EAC000120EBE63F8010FE0F030F0010000240F4
:101EBC002800024008540258F8ABFDA7CDCCCCCC7E
:101ECC00F0B583B0044600230193894B1D68894B00
:101EDC00A3FB0535AD0A876D3E68D7F800C00368D3
:101EEC0085498648834218BF8B420CBF01200020D5
:101EFC0079D0834A934276D01832934273D01832F9
:101F0C00934270D0183293426DD0183293426AD0FB
:101F1C001832934267D002F55672934263D018324E
:101F2C00934260D0183293425DD0183293425AD00B
:101F3C001832934257D01832934254D018329342ED
:101F4C0051D0183293424ED06E496F4A934218BF0B
:101F5C008B422AD06D4A934227D01432934224D01C
:101F6C001432934221D0143293421ED01432934235
:101F7C001BD01432934218D0654A934215D01432B8
:101F8C00934212D0143293420FD0143293420CD09D
:101F9C001432934209D01432934206D01432934235
:101FAC0003D01432934240F061821A68E16D01F063
:101FBC001F010420884010EA0C0F00F0A78212F0D9
:101FCC00040F00F0A382786012F4004F00F05A82E4
:101FDC0012F4803F40F05082A36C002B00F046823C
:101FEC002046984742E2E26D02F01F0108228A4027
:101FFC00324241D070BB424A93422BD018329342AA
:10200C0028D01832934225D01832934222D018325D
:10201C0093421FD0183293421CD002F55672934251
:10202C0018D01832934215D01832934212D018326D
:10203C0093420FD0183293420CD01832934209D0ED
:10204C001832934206D01832934203D01A68C2F366
:10205C00C00202E01A68C2F380026AB11A6822F068
:10206C0004021A60E36D03F01F0208239340BB6067
:10207C00636D43F001036365E26D02F01F0226FA03
:10208C0002F313F0010F49D023681B481B498B4204
:10209C0018BF83423ED018318B423BD018318B4253
:1020AC0038D018318B4235D018318B4232D01831A0
:1020BC008B422FD018318B422CD001F556718B42AC
:1020CC0028D018318B4225D018318B4222D01831B0
:1020DC008B421FD018318B421CD018318B4219D037
:1020EC0018318B4216D018318B4213D01B6815E077
:1020FC000C000020B5814E1B10000240280002404D
:10210C0040000240082C02481C2C0248302C02488B
:10211C00085402585B6913F0800F3BD1E36D03F058
:10212C001F03042202FA03F333423FD0226895487E
:10213C0095498A4218BF824234D018318A4231D034
:10214C0018318A422ED018318A422BD018318A424B
:10215C0028D018318A4225D018318A4222D001F574
:10216C0056718A421ED018318A421BD018318A42CD
:10217C0018D018318A4215D018318A4212D0183131
:10218C008A420FD018318A420CD018318A4209D0B9
:10219C0013680BE001239340BB60636D43F00203B3
:1021AC006365BBE7126812F0020F3DD1E36D03F0DB
:1021BC001F03102202FA03F333425FD022687148E6
:1021CC0071498A4218BF824234D018318A4231D0C8
:1021DC0018318A422ED018318A422BD018318A42BB
:1021EC0028D018318A4225D018318A4222D001F5E4
:1021FC0056718A421ED018318A421BD018318A423D
:10220C0018D018318A4215D018318A4212D01831A0
:10221C008A420FD018318A420CD018318A4209D028
:10222C001268C2F3800208E0BB60636D43F00403E4
:10223C006365BBE71268C2F3C002FAB1BB602368E6
:10224C001A6812F4802F0DD01B6813F4002F04D1E0
:10225C00236C9BB12046984710E0A36C73B12046C9
:10226C0098470BE01A6812F4807F03D11A6822F0A9
:10227C0008021A60236C0BB120469847E36D03F0FB
:10228C001F03202202FA03F3334200F091802268EC
:10229C003C483D498A4218BF82422ED018318A42AE
:1022AC002BD018318A4228D018318A4225D01831C7
:1022BC008A4222D018318A421FD018318A421CD04F
:1022CC0001F556718A4218D018318A4215D018314E
:1022DC008A4212D018318A420FD018318A420CD05F
:1022EC0018318A4209D018318A4206D018318A42F4
:1022FC0003D01268C2F3400202E01268C2F300126B
:10230C00002A55D0BB6094F83530042B0ED02368CE
:10231C001A6812F4802F39D01B6813F4002F2CD1BB
:10232C00636C002B44D02046984741E02268136828
:10233C0023F0160313602268536923F08003536162
:10234C00236CB3B12268136823F008031360E36DA8
:10235C0003F01F023F239340BB60012384F8353008
:10236C00002384F83430236D002B7FD0204698470F
:10237C007CE0A36C002BE5D1E9E7E36BC3B120460D
:10238C00984715E010000240280002401A6812F429
:10239C00807F09D11A6822F010021A60012384F898
:1023AC003530002384F83430E36B0BB1204698476A
:1023BC00636D002B5AD0636D13F0010F52D00423C0
:1023CC0084F8353023689649964A934218BF8B425D
:1023DC002FD0183293422CD01832934229D0183275
:1023EC00934226D01832934223D01832934220D0F5
:1023FC00183293421DD002F55672934219D01832FE
:10240C00934216D01832934213D01832934210D004
:10241C00183293420DD0183293420AD0183293429C
:10242C0007D01832934204D01A6822F001021A60C5
:10243C0003E01A6822F001021A60019B0133019338
:10244C00AB4204D823681B6813F0010FF5D1236845
:10245C001B6813F0010F0BD0032384F835300023D5
:10246C0084F83430E36C0BB12046984703B0F0BDD0
:10247C00012384F83530F2E7236C002BF6D020468C
:10248C009847F3E712F0200F3AD123686449654A64
:10249C00934218BF8B422FD0183293422CD0183253
:1024AC00934229D01832934226D01832934223D02B
:1024BC001832934220D0183293421DD002F5567236
:1024CC00934219D01832934216D01832934213D03B
:1024DC001832934210D0183293420DD018329342D6
:1024EC000AD01832934207D01832934204D01A689B
:1024FC0022F004021A6003E01A6822F008021A6043
:10250C00236C002BB2D020469847AFE702208840BE
:10251C0010EA0C0F60D012F0020F5DD0786012F44C
:10252C00004F0ED012F4803F05D1636C002B9DD070
:10253C00204698479AE7E36B002B97D020469847A4
:10254C0094E712F0200F40D123683549354A934265
:10255C0018BF8B422FD0183293422CD01832934292
:10256C0029D01832934226D01832934223D01832F5
:10257C00934220D0183293421DD002F556729342EA
:10258C0019D01832934216D01832934213D0183205
:10259C00934210D0183293420DD0183293420AD085
:1025AC001832934207D01832934204D01A6822F0A2
:1025BC000A021A6003E01A6822F014021A6001235E
:1025CC0084F83530002384F83430E36B002B3FF46F
:1025DC004DAF2046984749E7082000FA01F111EA6F
:1025EC000C0F3FF443AF12F0080F3FF43FAF1A68E3
:1025FC0022F00E021A60E36D03F01F03012202FAAF
:10260C0003F37B60626584F83520002384F8343052
:10261C00E36C002B3FF42AAF2046984726E700BF17
:10262C00100002402800024030B4416B0468D4F81A
:10263C0084306F4A134043EA8103C4F88430046841
:10264C00D4F8843023F47F03856B43EA0543C4F844
:10265C008430836B0B440468D4F88810114041EA31
:10266C008301C4F888100468D4F8881021F4FE01A2
:10267C00C56B41EA0541C4F88810C16B03EB4103FB
:10268C000468D4F8A010114041EA8301C4F8A010EA
:10269C000468D4F8A01021F4FE01056C41EA054150
:1026AC00C4F8A010016C446C04FB01330468D4F82A
:1026BC00B010114041EA8301C4F8B0100468D4F89A
:1026CC00B01021F4FE01856C41EA0541C4F8B0104C
:1026DC00816CC46C04FB01330468D4F8AC10114059
:1026EC0041EA8301C4F8AC10016D446D04FB013365
:1026FC000468D4F8F010114041EA8301C4F8F010DA
:10270C000468D4F8F01021F47C11856D41EA054180
:10271C00C4F8F010816D03EB41030468D4F8C010C9
:10272C000A4042EA8303C4F8C0300268D2F8C030D1
:10273C0023F47C13C16D43EA0143C2F8C030026834
:10274C00D2F8C03023F07C53016E43EA0163C2F827
:10275C00C030436B274A1A449200C266836B02EB6B
:10276C0083030367C16B03EBC1034367016C446CC8
:10277C0004FB01F103EB81038367816CC46C04FBE4
:10278C0001F103EB8103C367016D446D04FB01F19F
:10279C0003EB8103C0F88030816D03EBC103C0F8FB
:1027AC008430816EC46D01FB04FC03EB8C03C0F818
:1027BC008830046E04FB01F103EB8103C0F8903008
:1027CC000D498B420DD9D0F89C3043F02003C0F852
:1027DC009C30032380F89830012007E0002342F856
:1027EC00043BD0F890309342F8D8002030BC7047AE
:1027FC000300FFFF002B0010FCD3004030B595B058
:10280C0004464C22A04901A803F08CFD002C00F0DA
:10281C00388123689D4A934220D094F898300BB3AA
:10282C002268936923F010039361FEF791F9054632
:10283C0023689A6912F0080F1AD0FEF789F9431B26
:10284C000A2BF5D9D4F89C3043F00103C4F89C3022
:10285C00032384F89830012015B030BD03F5807344
:10286C006360DAE784F89930204600F0E5FAD7E7A0
:10287C009A6942F001029A61FEF76AF905462368EB
:10288C009A6912F0010F0FD1FEF762F9401B0A286A
:10289C00F5D9D4F89C3043F00103C4F89C300323E1
:1028AC0084F898300120D7E79A6942F002029A61C5
:1028BC00237C012B40D02268936943F04003936141
:1028CC00637C012B3ED02268936923F4804393618F
:1028DC00A37C012B3CD02268936943F48053936111
:1028EC002268936923F44073A1680B4393612268B7
:1028FC00936923F0A40393612268136923F01003F6
:10290C001361E368012B29D0002B2CD0022B00F093
:10291C009B802268936943F080039361226813695A
:10292C0043F010031361E368032B1CD122689369F5
:10293C0043F02003936116E02268936923F040036F
:10294C009361BDE72268936943F480439361BFE7C9
:10295C002268936923F480539361C1E722689369D9
:10296C0043F004039361A3695A1EE369013B1B0204
:10297C0043EA4263226A013A13436269013A2168CD
:10298C0043EA0243CB61A368B3F5407F62D0236E68
:10299C0033B12268D2F8C030616E0B43C2F8C0303C
:1029AC00E36D226ED3420DD02168D1F8C83023F0EC
:1029BC000703A26E14A800EB820252F84C2C1343AE
:1029CC00C1F8C830236C6BB12168D1F8BC3023F04E
:1029DC000703626C14A800EB820252F84C2C1343D0
:1029EC00C1F8BC30A36C73B12168D1F8BC3023F0B2
:1029FC007003E26C14A800EB820252F84C2C43EAF0
:102A0C000213C1F8BC30236D73B12168D1F8BC300E
:102A1C0023F4E063626D14A800EB820252F84C2C94
:102A2C0043EA0223C1F8BC302268184B9A4222D0E8
:102A3C000023C4F89430C4F89C30012384F89830F7
:102A4C002046FFF7F1FD07E72268936943F0200366
:102A5C00936188E7A36A013BE26A013A43EA0223E5
:102A6C00226B013A43EA0213626A013A216843EA93
:102A7C000243CB608BE76268936823F00303936097
:102A8C00D6E70120E8E600BF6463000800A0004020
:102A9C00F0B583B000236BE085685E000324B4407E
:102AAC0025EA0405CC68B4402C438460456825EACB
:102ABC000C054C68C4F300149C402C43446069E042
:102ACC00DD08083550F8254003F0070C4FEA8C0C54
:102ADC004FF00F0E0EFA0CFE24EA0E0E0C6904FADF
:102AEC000CF444EA0E0440F825406BE0092400E0A5
:102AFC00002404FA0EF42C430CF1020C694D45F839
:102B0C002C404FF0B0442568D44325EA02064F68A8
:102B1C0017F4801F01D042EA05064FF0B0452E6035
:102B2C006D6804EA05064F6817F4001F01D042EAED
:102B3C0005064FF0B0456E60D5F8845004EA0506E2
:102B4C004F6817F4003F01D042EA05064FF0B0453C
:102B5C00C5F88460D5F880502C404E6816F4803F40
:102B6C0001D042EA05044FF0B042C2F88040013374
:102B7C000A6832FA03F400F092804FF0010C0CFA60
:102B8C0003FC1CEA0202F2D04C6804F00304013C82
:102B9C00012C81D94C6804F00304032C0CD0C468BC
:102BAC005D004FF0030C0CFA05FC24EA0C0C8C684D
:102BBC00AC4044EA0C04C4604C6804F00304022CDE
:102BCC003FF47EAF04684FEA430E4FF0030C0CFA4F
:102BDC000EFC24EA0C0C4C6804F0030404FA0EF40A
:102BEC0044EA0C0404604C6814F4403FBFD02E4CF3
:102BFC00D4F8545145F00205C4F85451D4F854415A
:102C0C0004F002040194019C4FEA930C0CF10205B0
:102C1C00244C54F8255003F0030E4FEA8E0E0F246B
:102C2C0004FA0EF425EA0405204CA0423FF460AFF0
:102C3C0004F58064A04222D004F58064A04220D028
:102C4C0004F58064A0421ED004F58064A0421CD020
:102C5C0004F58064A0421AD004F58064A04218D018
:102C6C0004F58064A04216D004F58064A04214D010
:102C7C0004F58064A0423FF439AF0A2439E70124FB
:102C8C0037E7022435E7032433E7042431E705242E
:102C9C002FE706242DE707242BE7082429E703B0A8
:102CAC00F0BD00BF00040058004402580000025858
:102CBC000AB18161704709048161704782B0074B8A
:102CCC00D3F8542142F00202C3F85421D3F8543102
:102CDC0003F002030193019B02B0704700440258B9
:102CEC00F0B5BBB00446002135913691379138913F
:102CFC003991C02204A803F0E8FA2268474B9A42A3
:102D0C0001D03BB0F0BD4FF400220023CDE90423E9
:102D1C0002230693142207920C22089209930A9319
:102D2C00C0230B9304A801F00FF9002870D13C4B81
:102D3C00D3F8382142F02002C3F83821D3F83821D7
:102D4C0002F020020092009AD3F8402142F00402D3
:102D5C00C3F84021D3F8402102F004020192019AF9
:102D6C00D3F8402142F00102C3F84021D3F84021AE
:102D7C0002F001020292029AD3F8402142F00202C0
:102D8C00C3F84021D3F8403103F002030393039BB3
:102D9C003F233593032636960025379535AF3946B4
:102DAC002048FFF775FEFF23359336963795394645
:102DBC001D48FFF76DFE35963696379539461B48FC
:102DCC00FFF766FE1A481B4B0360092343608560BE
:102DDC00C5604FF4806303614FF4006343614FF4AB
:102DEC00005383614FF48073C3614FF480330362EB
:102DFC004562FEF775FE70B90D4BE3649C630022CF
:102E0C0011461220FEF7C4FC1220FEF7D1FC78E725
:102E1C00FDF748FB8BE7FDF745FBEDE70020024093
:102E2C0000440258000802580000025800040258DE
:102E3C00E80200201000024010B5BAB00446002190
:102E4C0035913691379138913991C02204A803F00D
:102E5C003CFA23683F4A934204D03F4A93423DD008
:102E6C003AB010BD4FF400420023CDE9042304A86E
:102E7C0001F06AF808BB394A136801331360012B5F
:102E8C001ED0374BD3F8402142F00202C3F8402148
:102E9C00D3F8403103F002030193019B4FF44073CC
:102EAC0035930223369300233793389309233993B0
:102EBC0035A92C48FFF7ECFDD2E7FDF7F3FADAE77A
:102ECC00274BD3F84C2142F48072C3F84C21D3F831
:102EDC004C3103F480730093009BD2E74FF4004213
:102EEC000023CDE9042304A801F02EF808BB1B4AEB
:102EFC00136801331360012B1ED0194BD3F84021FA
:102F0C0042F00202C3F84021D3F8403103F002032F
:102F1C000393039B4FF440533593022336930023C2
:102F2C00379338930923399335A90E48FFF7B0FD31
:102F3C0096E7FDF7B7FADAE7094BD3F84C2142F4E0
:102F4C008072C3F84C21D3F84C3103F48073029394
:102F5C00029BD2E700A0004000A40040C803002060
:102F6C00004402580004025882B00368114A93428C
:102F7C0004D0114A93420FD002B070470F4BD3F8D4
:102F8C00502142F00102C3F85021D3F8503103F024
:102F9C0001030093009BEFE7084BD3F8482142F064
:102FAC001002C3F84821D3F8483103F01003019301
:102FBC00019BE1E700000140001000400044025872
:102FCC0082B00368114A934204D0114A93420FD045
:102FDC0002B070470F4BD3F8482142F00202C3F8FD
:102FEC004821D3F8483103F002030093009BEFE72C
:102FFC00084BD3F8482142F00402C3F84821D3F817
:10300C00483103F004030193019BE1E70004004005
:10301C00000800400044025800B589B00023039317
:10302C000493059306930793026803F1804303F519
:10303C0082339A4202D009B05DF804FB114BD3F8ED
:10304C00502142F00202C3F85021D3F8502102F073
:10305C0002020192019AD3F8402142F00402C3F813
:10306C004021D3F8403103F004030293029BC023A8
:10307C000393022304930323079303A90248FFF746
:10308C0007FDD8E7004402580008025830B58BB051
:10309C000023059306930793089309930368354A15
:1030AC00934207D0344A93421DD0344A93424AD0BB
:1030BC000BB030BD324BD3F8402142F00102C3F8C3
:1030CC004021D3F8403103F001030193019B4FF4ED
:1030DC0070630593022306930123099305A92948DC
:1030EC00FFF7D6FCE4E7264BD3F8402142F004026C
:1030FC00C3F84021D3F8402102F004020292029A54
:10310C00D3F8402142F00202C3F84021D3F84031F9
:10311C0003F002030393039B4FF400730593022403
:10312C000694099405AD29461748FFF7B1FC2023F6
:10313C000593069400230793089309942946134892
:10314C00FFF7A6FCB4E70E4BD3F8402142F0020285
:10315C00C3F84021D3F8403103F002030493049BDD
:10316C00C023059302230693099305A90748FFF78B
:10317C008FFC9DE700000140000400400008004067
:10318C00004402580000025800080258000402587B
:10319C00134BDB6813F0040F07D1114BDB6803F002
:1031AC00070383421AD00120704710B50C4AD3682C
:1031BC0023F007030343D360FDF7CAFC0446084B16
:1031CC005B6813F4005F07D1FDF7C2FC001BB0F580
:1031DC007A7FF4D9012000E0002010BD0020704758
:1031EC0000480258002800F0118338B504460368E3
:1031FC0013F0010F29D0A14A136903F03803926A26
:10320C00102B19D0182B13D06368B3F5803F43D023
:10321C00002B58D1994B1A6822F480321A601A6824
:10322C0022F480121A601A6822F480221A6038E0A4
:10323C0002F00302022AE7D1904B1B6813F4003F03
:10324C0003D06368002B00F0E382236813F0020FB5
:10325C0000F0A280894A1369926A13F0380374D083
:10326C00182B6FD0E368002B00F0C38083490A68E9
:10327C0022F0190213430B60FDF76AFC05467F4BE5
:10328C001B6813F0040F40F0AB80FDF761FC401B92
:10329C000228F4D90320C2E2784A136843F480333D
:1032AC0013606368002B3ED0FDF752FC0546734B50
:1032BC001B6813F4003FC8D1FDF74AFC401B64287F
:1032CC00F5D90320ABE2B3F5A02F10D0B3F5A81FAE
:1032DC001BD06A4B1A6822F480321A601A6822F4E6
:1032EC0080221A601A6822F480121A60D9E7634BA4
:1032FC001A6842F480221A601A6822F480121A604A
:10330C001A6842F480321A60CBE75C4B1A6842F4BC
:10331C0080221A601A6842F480121A601A6842F409
:10332C0080321A60BDE7FDF713FC0546534B1B6852
:10333C0013F4003F89D0FDF70BFC401B6428F5D932
:10334C0003206CE212F0030F8CD14C4B1B6813F072
:10335C00040F03D0E368002B00F05C82474A13682B
:10336C0023F01903E1680B431360FDF7F1FB0546ED
:10337C00424B1B6813F0040F06D1FDF7E9FB401B11
:10338C000228F5D903204AE23C4A536823F0FE4355
:10339C00216943EA01635360236813F0100F51D085
:1033AC00364A136903F03803926A082B39D0182B6C
:1033BC0033D0E369002B6CD0304A136843F08003A0
:1033CC001360FDF7C5FB05462C4B1B6813F4807F7F
:1033DC0056D1FDF7BDFB401B0228F5D903201EE298
:1033EC00264A536823F0FE43216943EA0163536084
:1033FC00D2E7224A136823F001031360FDF7A8FB00
:10340C0005461E4B1B6813F0040FC5D0FDF7A0FB3F
:10341C00401B0228F5D9032001E202F00302012A25
:10342C00C7D1164B1B6813F4807F03D0E369802B44
:10343C0040F0F281114AD36823F07C53216A43EAAD
:10344C000163D360236813F0080F4AD06369002B23
:10345C0033D00A4A536F43F001035367FDF778FBEF
:10346C000546064B5B6F13F0020F3AD1FDF770FB6C
:10347C00401B0228F5D90320D1E100BF00440258BB
:10348C008C4AD36823F07C53216A43EA0163D360EE
:10349C00D8E7884A136823F080031360FDF758FBC4
:1034AC000546844B1B6813F4807FCBD0FDF750FB93
:1034BC00401B0228F5D90320B1E17E4A536F23F05B
:1034CC0001035367FDF744FB05467A4B5B6F13F022
:1034DC00020F06D0FDF73CFB401B0228F5D9032058
:1034EC009DE1236813F0200F29D0A3699BB1714A89
:1034FC00136843F480531360FDF72AFB05466D4BAC
:10350C001B6813F4005F1AD1FDF722FB401B022845
:10351C00F5D9032083E1674A136823F480531360C1
:10352C00FDF716FB0546634B1B6813F4005F06D0D2
:10353C00FDF70EFB401B0228F5D903206FE1236831
:10354C0013F0040F22D1636A002B00F06781594AF3
:10355C00126902F03802182A00F00E81022B00F0DA
:10356C009480544A136823F080731360FDF7F0FACB
:10357C000446504B1B6813F0007F00F0FB80FDF7F6
:10358C00E7FA001B0228F4D9032048E14A4A1368E1
:10359C0043F480731360FDF7DBFA0546464B1B685A
:1035AC0013F4807F06D1FDF7D3FA401B6428F5D9BC
:1035BC00032034E1A368012B0ED033BB3D4B1A6FB3
:1035CC0022F001021A671A6F22F080021A671A6F32
:1035DC0022F004021A6704E0364A136F43F0010329
:1035EC001367A368002B3ED0FDF7B2FA0546314BAA
:1035FC001B6F13F0020FA6D1FDF7AAFA401B41F284
:10360C0088339842F3D9032009E1052B0FD0852B81
:10361C001BD0284B1A6F22F001021A671A6F22F086
:10362C0004021A671A6F22F080021A67D9E7214B3D
:10363C001A6F42F004021A671A6F22F080021A679E
:10364C001A6F42F001021A67CBE71A4B1A6F42F05D
:10365C0004021A671A6F42F080021A671A6F42F05E
:10366C0001021A67BDE7FDF773FA0546114B1B6F94
:10367C0013F0020F3FF467AFFDF76AFA401B41F2FB
:10368C0088339842F2D90320C9E00A4A136823F020
:10369C0080731360FDF75CFA0546064B1B6813F04C
:1036AC00007F0BD0FDF754FA401B0228F5D90320FC
:1036BC00B5E000BF00440258004802585F4B996ABD
:1036CC005F4A0A40A16AE06A41EA00110A439A6221
:1036DC00226B013AC2F30802616B0139490289B2CB
:1036EC000A43A16B0139090401F4FE010A43E16BA1
:1036FC000139090601F0FE410A431A63DA6A22F025
:10370C000102DA625A6B6FF3CF02A16C42EAC1027A
:10371C005A63DA6A22F00C02216C0A43DA62DA6A22
:10372C0022F00202616C0A43DA62DA6A42F48032F5
:10373C00DA62DA6A42F40032DA62DA6A42F480223D
:10374C00DA62DA6A42F00102DA621A6842F08072D6
:10375C001A60FDF7FDF90446384B1B6813F0007F27
:10376C0006D1FDF7F5F9001B0228F5D9032056E028
:10377C00002054E0002052E030498A6A086B012B8B
:10378C004ED002F00303A16A8B424BD1C2F3051257
:10379C00E36A9A4248D1C0F30802236B013B9A4278
:1037AC0044D1C0F34622636B013B9A4240D1C0F333
:1037BC000642A36B013B9A423CD1C0F30660E36B1B
:1037CC00013B984238D11D4B5B6BC3F3CC03A26C0D
:1037DC009A4201D1002022E0184AD36A23F0010357
:1037EC00D362FDF7B5F90546FDF7B2F9A842FBD057
:1037FC00124A536B6FF3CF03A16C43EAC1035363BB
:10380C00D36A43F00103D362002008E00120704723
:10381C00012004E0012002E0012000E0002038BD7E
:10382C000120FCE70120FAE70120F8E70120F6E788
:10383C000120F4E70120F2E70120F0E700440258F0
:10384C000CFCFFFF754B1B6903F03803102B00F0C9
:10385C00DE80182B0FD0002B40F0DB806F4B1B68E9
:10386C0013F0200F00F0D7806C4B1B68C3F3C1031F
:10387C006B48D840704710B4684B9A6A02F0030248
:10388C009C6AC4F30510D96A01F001015B6BC3F3A8
:10389C00CC0301FB03F307EE903AF8EE677A14F4CD
:1038AC007C7F77D0012A4AD0022A76D0002A40F0B9
:1038BC0091805A4B1B6813F0200F23D057490A688C
:1038CC00C2F3C102564BD34007EE103AF8EE476AEA
:1038DC0007EE100AB8EE476A86EE867A0B6BC3F3D6
:1038EC00080306EE903AF8EE666A9FED4E6A67EEB4
:1038FC00867A76EEA77AF7EE006A77EEA67A27EE4E
:10390C00277A38E007EE100AF8EE476A9FED466A10
:10391C0086EE267A414B1B6BC3F3080306EE903AF6
:10392C00F8EE666A9FED3F6A67EE867A76EEA77AC6
:10393C00F7EE006A77EEA67A27EE277A1BE007EE01
:10394C00100AF8EE476A9FED396A86EE267A334BF9
:10395C001B6BC3F3080306EE903AF8EE666A9FED14
:10396C00316A67EE867A76EEA77AF7EE006A77EE22
:10397C00A67A27EE277A294B1B6BC3F34623013318
:10398C0007EE903AF8EE677AC7EE276AFCEEE67A15
:10399C0017EE900A5DF8044B704707EE100AF8EE2C
:1039AC00476A9FED236A86EE267A1C4B1B6BC3F38A
:1039BC00080306EE903AF8EE666A9FED1A6A67EE17
:1039CC00867A76EEA77AF7EE006A77EEA67A27EE7D
:1039DC00277AD0E707EE100AF8EE476A9FED136AD4
:1039EC0086EE267A0D4B1B6BC3F3080306EE903A5A
:1039FC00F8EE666A9FED0B6A67EE867A76EEA77A2A
:103A0C00F7EE006A77EEA67A27EE277AB3E7094835
:103A1C007047094870470248704700BF004402587D
:103A2C000090D003000000390024744C0024744A28
:103A3C00001BB74B00366E0100093D00002800F05A
:103A4C00328170B50D4604469B4B1B6803F00F0387
:103A5C008B420BD2984A136823F00F030B4313606D
:103A6C00136803F00F038B4240F01F81236813F09F
:103A7C00040F0CD02269914B9B6903F070039A429E
:103A8C0005D98E498B6923F070031A438A61236828
:103A9C0013F0080F0CD06269884BDB6903F07003DC
:103AAC009A4205D98549CB6923F070031A43CA6140
:103ABC00236813F0100F0CD0A269804BDB6903F460
:103ACC00E0639A4205D97D49CB6923F4E0631A433C
:103ADC00CA61236813F0200F0CD0E269774B1B6A84
:103AEC0003F070039A4205D974490B6A23F07003F2
:103AFC001A430A62236813F0020F0CD0E2686F4B72
:103B0C009B6903F00F039A4205D96C498B6923F02A
:103B1C000F031A438A61236813F0010F41D0674ADF
:103B2C00936923F47063A1680B4393616368022B60
:103B3C000AD0032B27D0012B2CD0604A126812F02C
:103B4C00040F06D10120ADE0126812F4003F00F022
:103B5C00AE805A490A6922F0070213430B61FCF745
:103B6C00F7FF0646554B1B6903F038036268B3EB4D
:103B7C00C20F16D0FCF7ECFF801B41F28833984241
:103B8C00F0D903208EE04D4A126812F0007FE0D18C
:103B9C00012087E0494A126812F4807FD9D10120B4
:103BAC0080E0236813F0020F0CD0E268434B9B6952
:103BBC0003F00F039A4205D240498B6923F00F039F
:103BCC001A438A613C4B1B6803F00F03AB420AD9C2
:103BDC00394A136823F00F032B431360136803F067
:103BEC000F03AB4265D1236813F0040F0CD022698C
:103BFC00324B9B6903F070039A4205D22F498B69B3
:103C0C0023F070031A438A61236813F0080F0CD059
:103C1C0062692A4BDB6903F070039A4205D227498B
:103C2C00CB6923F070031A43CA61236813F0100F99
:103C3C000CD0A269214BDB6903F4E0639A4205D2F4
:103C4C001E49CB6923F4E0631A43CA61236813F05D
:103C5C00200F0CD0E269194B1B6A03F070039A42D7
:103C6C0005D216490B6A23F070031A430A62FFF758
:103C7C00E9FD12498B69C3F30323114AD35C03F0AA
:103C8C001F03D8408B6903F00F03D35C03F01F03B1
:103C9C0020FA03F30B4A13600B4B18600B4B18689C
:103CAC00FCF7F4FE70BD012070470120FAE70120FB
:103CBC00F8E70120F6E700BF00200052004402584C
:103CCC00B8630008080000200C000020040000204D
:103CDC0008B5FFF7B7FD0B4A9369C3F303230A49F1
:103CEC00CB5C03F01F0320FA03F3926902F00F027E
:103CFC00885C00F01F0023FA00F0044A1060044AAC
:103D0C00136008BD00440258B86300080800002086
:103D1C000C00002008B5FFF7DBFF054BDB69C3F394
:103D2C000213044AD35C03F01F03D84008BD00BF44
:103D3C0000440258B8630008404B9B6A03F003032D
:103D4C00032B79D070B505460E463C4A136823F018
:103D5C0080631360FCF7FCFE0446384B1B6813F0C1
:103D6C00006F06D0FCF7F4FE031B022BF5D90320E1
:103D7C0070BD324B9A6A22F47C32296842EA0132D5
:103D8C009A626A68013AC2F30802A96801394902C9
:103D9C0089B20A43E9680139090401F4FE010A43B6
:103DAC0029690139090601F0FE410A439A63DA6A6E
:103DBC0022F0C00269690A43DA62DA6A22F0200250
:103DCC00A9690A43DA62DA6A22F01002DA62DA6B63
:103DDC006FF3CF02E96942EAC102DA63DA6A42F0B0
:103DEC001002DA62C6B91A46DB6A43F40023D362C6
:103DFC00124A136843F080631360FCF7A9FE044673
:103E0C000E4B1B6813F0006F14D1FCF7A1FE001BC6
:103E1C000228F5D90320ABE7012E05D0074AD36A57
:103E2C0043F40013D362E3E7044AD36A43F48013E8
:103E3C00D362DDE700209BE7012070470044025865
:103E4C00404B9B6A03F00303032B79D070B50546F6
:103E5C000E463C4A136823F080531360FCF778FE3F
:103E6C000446384B1B6813F0005F06D0FCF770FE5D
:103E7C00031B022BF5D9032070BD324B9A6A22F03A
:103E8C007C72296842EA01529A626A68013AC2F36A
:103E9C000802A9680139490289B20A43E968013963
:103EAC00090401F4FE010A4329690139090601F0EC
:103EBC00FE410A431A64DA6A22F4406269690A43D1
:103ECC00DA62DA6A22F40072A9690A43DA62DA6AFF
:103EDC0022F48072DA625A6C6FF3CF02E96942EA1B
:103EEC00C1025A64DA6A42F48072DA62C6B91A46BE
:103EFC00DB6A43F48003D362124A136843F08053A5
:103F0C001360FCF725FE04460E4B1B6813F0005F94
:103F1C0014D1FCF71DFE001B0228F5D90320ABE7DA
:103F2C00012E05D0074AD36A43F08073D362E3E7CE
:103F3C00044AD36A43F40003D362DDE700209BE715
:103F4C000120704700440258F8B50446036813F08A
:103F5C00006F30D0C36EB3F5001F26D00ED8ABB1B6
:103F6C00B3F5801F07D102210830FFF7E5FE0546A7
:103F7C0095B12E4621E0012635461EE0B3F5401FD3
:103F8C0001D1002508E00126354616E0974AD36A90
:103F9C0043F40033D3620025944A136D23F4401389
:103FAC00E16E0B431365002607E002212830FFF772
:103FBC0047FF0546DCE700263546236813F4807F6F
:103FCC0014D0A36D042B31D8DFE803F003222908A9
:103FDC000800864AD36A43F40033D3624DBB834A4C
:103FEC00136D23F00703A16D0B431365236813F4C2
:103FFC00007F42D0E36D802B31D01FD84BB3402BC8
:10400C0019D1002104F10800FFF796FE05462CE0BB
:10401C00002104F10800FFF78FFE0546DEE70021C2
:10402C0004F12800FFF70CFF0546D7E701263546BB
:10403C00DCE72E46DAE7012635461EE0B3F5807F35
:10404C0013D0B3F5A07F10D0C02B0ED0012635466F
:10405C0013E0664AD36A43F40033D36205E00021CF
:10406C0004F12800FFF7ECFE0546D5B95F4A136D45
:10407C0023F4E073E16D0B431365236813F4806F35
:10408C0034D0236EB3F5806F22D00FD8D3B1B3F5F3
:10409C00007F08D1002104F10800FFF74DFE054612
:1040AC001CE02E46E9E7012635461FE0B3F5006F0C
:1040BC0014D0B3F5206F11D0B3F5C06F0ED001261C
:1040CC00354613E0494AD36A43F40033D36205E022
:1040DC00002104F12800FFF7B3FE0546BDB9434AA1
:1040EC00136D23F46063216E0B431365236813F087
:1040FC00007F24D0E36C202B13D00DD8BBB1102B38
:10410C0007D13A4AD36A43F40033D3620FE02E4608
:10411C00ECE70126354612E0302B08D00126354657
:10412C000DE0022104F10800FFF706FE0546D5B9A3
:10413C002E4AD36C23F03003E16C0B43D364236819
:10414C0013F4805F31D0636EB3F5005F1FD00FD8CE
:10415C00BBB1B3F5805F08D1002104F10800FFF773
:10416C00EBFD054619E02E46E9E7012635461CE035
:10417C00B3F5405F11D0B3F5804F0ED00126354614
:10418C0013E01A4AD36A43F40033D36205E00021EA
:10419C0004F12800FFF754FE054615BB134A136DB6
:1041AC0023F4E043616E0B431365236813F4005F43
:1041BC0032D0A36EB3F5003F26D019D843B1B3F576
:1041CC00803F10D1012104F10800FFF7B5FD054631
:1041DC000DBB064A136D23F4E023A16E0B4313654C
:1041EC001AE02E46E1E70126354615E00044025858
:1041FC00B3F5802FECD0B3F5A02FE9D0B3F5403F49
:10420C00E6D00126354607E0012104F12800FFF72E
:10421C0017FE0546DCE72E46236813F4804F18D0B2
:10422C00D4F8B030B3F1005F38D024D843B1B3F137
:10423C00805F1DD1012104F10800FFF77DFD0546CB
:10424C009DBB904A936D23F0E043D4F8B0100B4320
:10425C009365236813F4004F3FD0A36FB3F1805FD5
:10426C0025D0B3F1005F30D033B30126354634E0AE
:10427C0001263546EDE7B3F1A04FE1D008D8B3F1F4
:10428C00405FDDD0B3F1804FDAD001263546E0E750
:10429C00B3F1C04FD4D001263546DAE7012104F141
:1042AC002800FFF7CDFD0546CAE72E46D1E7754A33
:1042BC00D36A43F40033D36275B9724A136D23F099
:1042CC004053A16F0B43136507E0012104F1080073
:1042DC00FFF732FD0546EFE72E46236813F0807F8B
:1042EC0013D0A36C032B3CD8DFE803F00702340790
:1042FC00644AD36A43F40033D362ADBB614AD36CD6
:10430C0023F00303A16C0B43D364236813F4800FD5
:10431C002CD1236813F0010F00F0A580D4F8843061
:10432C00282B00F29E80DFE803F08B9C9C9C9C9CCD
:10433C009C9C859C9C9C9C9C9C9C959C9C9C9C9CCF
:10434C009C9C8B9C9C9C9C9C9C9C8B9C9C9C9C9CC3
:10435C009C9C8B00022104F10800FFF7EDFC054644
:10436C00CBE701263546D0E72E46CEE7464A136802
:10437C0043F480731360FCF7EBFB0746424B1B685E
:10438C0013F4807F05D1FCF7E3FBC01B6428F5D93F
:10439C000325002D4AD13B4B1B6FD4F8B42053405E
:1043AC0013F4407F0CD0374B1A6F22F44072196F04
:1043BC0041F480311967196F21F4803119671A673C
:1043CC00D4F8B430B3F5807F15D08DBBD4F8B430AD
:1043DC0003F44072B2F5407F1ED02A4A136923F4CD
:1043EC007C53136127490B6FD4F8B420C2F30B0232
:1043FC0013430B678DE7FCF7ABFB0746214B1B6F99
:10440C0013F0020FE1D1FCF7A3FBC01B41F2883380
:10441C009842F3D90325D8E71A48026922F47C5252
:10442C001A4901EA131313430361DBE72E4670E7C5
:10443C002E466EE7012104F10800FFF77DFC0546CE
:10444C00F5B9104A536D23F03803D4F884100B439C
:10445C00536508E0012104F12800FFF7F1FC054643
:10446C00EEE701263546236813F0020F1FD0D4F86F
:10447C008030052B33D8DFE803F0110B2B11111111
:10448C002E46F0E70044025800480258CFFFFF00C8
:10449C00012104F10800FFF74FFC054615BBB74A94
:1044AC00536D23F00703D4F880100B435365236836
:1044BC0013F0040F29D0D4F89C30052B00F208819E
:1044CC00DFE813F018001200FF00180018001800A5
:1044DC00012104F12800FFF7B3FC0546DEE70126B5
:1044EC003546E4E72E46E2E7012104F10800FFF728
:1044FC0023FC0546002D40F0EE80A04A936D23F07E
:10450C000703D4F89C100B439365236813F0200F1A
:10451C001DD0D4F89830B3F1005F00F0F08000F2B9
:10452C00DF804BB1B3F1805F40F0D780002104F104
:10453C000800FFF701FC0546002D40F0E7808F4A8C
:10454C00536D23F0E043D4F898100B435365236864
:10455C0013F0400F1DD0D4F8A430B3F5006F00F069
:10456C00E98000F2D8804BB1B3F5806F40F0D08079
:10457C00002104F10800FFF7DFFB0546002D40F099
:10458C00E0807E4A936D23F4E053D4F8A4100B43DF
:10459C009365236813F0800F1DD0D4F8A830B3F5C1
:1045AC00804F00F0E28000F2D1804BB1B3F5005F98
:1045BC0040F0C980002104F10800FFF7BDFB05465F
:1045CC00002D40F0D9806D4A936D23F46043D4F8EC
:1045DC00A8100B439365236813F0080F0DD0D4F883
:1045EC008C30B3F5805F00F0CB80644A536D23F4BC
:1045FC004053D4F88C100B435365236813F0100F01
:10460C000DD0D4F8A030B3F5807F00F0C3805B4AA6
:10461C00936D23F44073D4F8A0100B439365236877
:10462C0013F4002F1CD0D4F8AC30B3F5803F00F05D
:10463C00BB80B3F5003F08D0002B40F0BC800021BC
:10464C0004F10800FFF778FB0546002D40F0B6801A
:10465C004A4A936D23F44033D4F8AC100B43936562
:10466C00236813F4802F1CD0D4F89030B3F5001FBE
:10467C0000F0A680B3F5401F08D0B3F5801F40F0C2
:10468C00A6803E4AD36A43F40033D362002D40F037
:10469C00A1803A4A536D23F44013D4F890100B4385
:1046AC005365236813F4803F00F0AC80236D002B1E
:1046BC0000F09280B3F5803F00F09C8001263546D7
:1046CC00A0E0012104F12800FFF7BAFB054611E731
:1046DC000126354619E72E4617E70126354636E7FB
:1046EC00B3F1804F3FF428AFB3F1A04F3FF424AFA8
:1046FC00B3F1405F3FF420AF0126354627E7022196
:10470C0004F12800FFF79CFB054615E72E461EE733
:10471C00012635463DE7B3F5805F3FF42FAFB3F587
:10472C00A05F3FF42BAFB3F5406F3FF427AF0126EA
:10473C0035462EE7022104F12800FFF781FB0546E0
:10474C001CE72E4625E70126354644E7B3F5004F16
:10475C003FF436AFB3F5204F3FF432AFB3F5C04F53
:10476C003FF42EAF0126354635E7022104F128002F
:10477C00FFF766FB054623E72E462CE7004402585C
:10478C00022104F12800FFF75BFB00283FF42DAF5A
:10479C0001262AE7022104F12800FFF751FB00282B
:1047AC003FF435AF012632E7022104F12800FFF770
:1047BC0047FB054649E70126354651E72E464FE7AC
:1047CC00012104F12800FFF73BFB05465EE70126BB
:1047DC00354666E72E4664E76F4AD36A43F40033E6
:1047EC00D36275B96C4AD36C23F48033216D0B43BF
:1047FC00D36407E0022104F10800FFF79DFA054697
:10480C00EFE72E46236813F0005F11D1236813F4F1
:10481C00003F28D0D4F88830B3F5807F14D010D95D
:10482C00B3F5007F15D0B3F5407F12D001261AE006
:10483C00022104F12800FFF703FB0028E6D0012633
:10484C00E4E733B101260EE0534AD36A43F4003354
:10485C00D362002D68D1504A536D23F44073D4F8C1
:10486C0088100B435365236813F4801F06D04A4A03
:10487C00136D23F00043E16F0B431365236813F4AE
:10488C00001F06D0444A136D23F08073216F0B4335
:10489C001365236813F4006F06D03F4A936D23F021
:1048AC000063616F0B439365236813F0804F09D04D
:1048BC00394B1A6922F400421A611A69D4F8B810FB
:1048CC000A431A612368002B06DA334AD36C23F0AF
:1048DC004053616D0B43D364236813F4000F07D06E
:1048EC002D4A536D23F44003D4F894100B435365B5
:1048FC00636813F0010F19D1636813F0020F1ED116
:10490C00636813F0040F23D1636813F0080F28D1E8
:10491C00636813F0100F2DD1636813F0200F32D1A0
:10492C0006B101263046F8BD2E469CE7002104F165
:10493C000800FFF701FA0028DED00646DCE701216B
:10494C0004F10800FFF7F8F90028D9D00646D7E79C
:10495C00022104F10800FFF7EFF90028D4D0064635
:10496C00D2E7002104F12800FFF76AFA0028CFD023
:10497C000646CDE7012104F12800FFF761FA002873
:10498C00CAD00646C8E7022104F12800FFF758FAFE
:10499C000028C5D00126C5E70044025808B5FFF72A
:1049AC0097F9054B1B6AC3F30213044AD35C03F05B
:1049BC001F03D84008BD00BF00440258B86300086C
:1049CC0010B4794B9A6A9C6AC4F3053CD96AC1F35A
:1049DC000011DB6BC3F3CC0301FB03F314F47C3F3A
:1049EC0000F0DD8002F0030207EE903AF8EE677AF1
:1049FC00012A4BD0022A00F09880002A40F0B280A5
:104A0C00694B1B6813F0200F23D067490A68C2F367
:104A1C00C102664BD34007EE103AF8EE476A07EE38
:104A2C0010CAB8EE476A86EE867A8B6BC3F308031E
:104A3C0006EE903AF8EE666A9FED5D6A67EE867A4E
:104A4C0076EEA77AF7EE006A77EEA67A27EE277A4B
:104A5C0038E007EE10CAF8EE476A9FED566A86EE0C
:104A6C00267A514B9B6BC3F3080306EE903AF8EE93
:104A7C00666A9FED4F6A67EE867A76EEA77AF7EE56
:104A8C00006A77EEA67A27EE277A1BE007EE10CAAB
:104A9C00F8EE476A9FED486A86EE267A424B9B6B8E
:104AAC00C3F3080306EE903AF8EE666A9FED406A8F
:104ABC0067EE867A76EEA77AF7EE006A77EEA67A3C
:104ACC0027EE277A384A936BC3F3462307EE903AC6
:104ADC00F8EE677AF7EE006A77EEA67A87EE276A29
:104AEC00BCEEC66A80ED006A936BC3F3064307EE17
:104AFC00903AF8EE677A77EEA67A87EE276ABCEEE4
:104B0C00C66A80ED016A936BC3F3066307EE903AB5
:104B1C00F8EE677A77EEA67AC7EE276AFCEEE66ABD
:104B2C00C0ED026A5DF8044B704707EE10CAF8EE50
:104B3C00476A9FED226A86EE267A1B4B9B6BC3F36A
:104B4C00080306EE903AF8EE666A9FED196A67EE76
:104B5C00867A76EEA77AF7EE006A77EEA67A27EEDB
:104B6C00277AAFE707EE10CAF8EE476A9FED126A94
:104B7C0086EE267A0C4B9B6BC3F3080306EE903A39
:104B8C00F8EE666A9FED0A6A67EE867A76EEA77A89
:104B9C00F7EE006A77EEA67A27EE277A92E70023E3
:104BAC00036043608360BDE7004402580090D0036B
:104BBC00000000390024744C0024744A001BB74BCD
:104BCC0010B4794B9A6A9C6AC4F3055CD96AC1F338
:104BDC0000215B6CC3F3CC0301FB03F314F07C7F6B
:104BEC0000F0DD8002F0030207EE903AF8EE677AEF
:104BFC00012A4BD0022A00F09880002A40F0B280A3
:104C0C00694B1B6813F0200F23D067490A68C2F365
:104C1C00C102664BD34007EE103AF8EE476A07EE36
:104C2C0010CAB8EE476A86EE867A0B6CC3F308039B
:104C3C0006EE903AF8EE666A9FED5D6A67EE867A4C
:104C4C0076EEA77AF7EE006A77EEA67A27EE277A49
:104C5C0038E007EE10CAF8EE476A9FED566A86EE0A
:104C6C00267A514B1B6CC3F3080306EE903AF8EE10
:104C7C00666A9FED4F6A67EE867A76EEA77AF7EE54
:104C8C00006A77EEA67A27EE277A1BE007EE10CAA9
:104C9C00F8EE476A9FED486A86EE267A424B1B6C0B
:104CAC00C3F3080306EE903AF8EE666A9FED406A8D
:104CBC0067EE867A76EEA77AF7EE006A77EEA67A3A
:104CCC0027EE277A384A136CC3F3462307EE903A43
:104CDC00F8EE677AF7EE006A77EEA67A87EE276A27
:104CEC00BCEEC66A80ED006A136CC3F3064307EE94
:104CFC00903AF8EE677A77EEA67A87EE276ABCEEE2
:104D0C00C66A80ED016A136CC3F3066307EE903A32
:104D1C00F8EE677A77EEA67AC7EE276AFCEEE66ABB
:104D2C00C0ED026A5DF8044B704707EE10CAF8EE4E
:104D3C00476A9FED226A86EE267A1B4B1B6CC3F3E7
:104D4C00080306EE903AF8EE666A9FED196A67EE74
:104D5C00867A76EEA77AF7EE006A77EEA67A27EED9
:104D6C00277AAFE707EE10CAF8EE476A9FED126A92
:104D7C0086EE267A0C4B1B6CC3F3080306EE903AB6
:104D8C00F8EE666A9FED0A6A67EE867A76EEA77A87
:104D9C00F7EE006A77EEA67A27EE277A92E70023E1
:104DAC00036043608360BDE7004402580090D00369
:104DBC00000000390024744C0024744A001BB74BCB
:104DCC0010B4794B9A6A9C6AC4F3051CD96A01F039
:104DDC0001015B6BC3F3CC0301FB03F314F47C7F85
:104DEC0000F0DD8002F0030207EE903AF8EE677AED
:104DFC00012A4BD0022A00F09880002A40F0B280A1
:104E0C00694B1B6813F0200F23D067490A68C2F363
:104E1C00C102664BD34007EE103AF8EE476A07EE34
:104E2C0010CAB8EE476A86EE867A0B6BC3F308039A
:104E3C0006EE903AF8EE666A9FED5D6A67EE867A4A
:104E4C0076EEA77AF7EE006A77EEA67A27EE277A47
:104E5C0038E007EE10CAF8EE476A9FED566A86EE08
:104E6C00267A514B1B6BC3F3080306EE903AF8EE0F
:104E7C00666A9FED4F6A67EE867A76EEA77AF7EE52
:104E8C00006A77EEA67A27EE277A1BE007EE10CAA7
:104E9C00F8EE476A9FED486A86EE267A424B1B6B0A
:104EAC00C3F3080306EE903AF8EE666A9FED406A8B
:104EBC0067EE867A76EEA77AF7EE006A77EEA67A38
:104ECC0027EE277A384A136BC3F3462307EE903A42
:104EDC00F8EE677AF7EE006A77EEA67A87EE276A25
:104EEC00BCEEC66A80ED006A136BC3F3064307EE93
:104EFC00903AF8EE677A77EEA67A87EE276ABCEEE0
:104F0C00C66A80ED016A136BC3F3066307EE903A31
:104F1C00F8EE677A77EEA67AC7EE276AFCEEE66AB9
:104F2C00C0ED026A5DF8044B704707EE10CAF8EE4C
:104F3C00476A9FED226A86EE267A1B4B1B6BC3F3E6
:104F4C00080306EE903AF8EE666A9FED196A67EE72
:104F5C00867A76EEA77AF7EE006A77EEA67A27EED7
:104F6C00277AAFE707EE10CAF8EE476A9FED116A91
:104F7C0086EE267A0C4B1B6BC3F3080306EE903AB5
:104F8C00F8EE666A9FED0A6A67EE867A76EEA77A85
:104F9C00F7EE006A77EEA67A27EE277A92E70023DF
:104FAC00036043608360BDE7004402580090D00367
:104FBC00000000390024744C0024744A001BB74BC9
:104FCC0000B58BB0A0F580730B4328D0A0F500730F
:104FDC000B4377D0A0F580630B4300F0CB80A0F59A
:104FEC0080530B4300F02381A0F500530B4300F0DA
:104FFC008381A0F500230B4300F0CC81A0F5803316
:10500C000B4300F00F82A0F580430B4300F0288285
:10501C00A0F50040084300F07D8200200CE0944B8A
:10502C001B6D03F00703042B00F29E82DFE803F0F4
:10503C0007111B0325008F480BB05DF804FB8C4B4C
:10504C00186810F00070F7D007A8FFF7B9FE0898A1
:10505C00F2E7874B186810F00060EDD004A8FFF75A
:10506C00AFFC0498E8E7824B186810F00050E3D0CE
:10507C0001A8FFF7A5FD0198DEE77D4AD36C03F08C
:10508C004053126812F0040F07D033B9784B1B68E9
:10509C00C3F3C1037848D840CEE7754A126812F4BE
:1050AC00807F03D0B3F1805F00F06082704A126899
:1050BC0012F4003F00F05C82B3F1005F00F05A8202
:1050CC000020B9E76A4B1B6D03F4E073802B31D0E1
:1050DC0015D9C02B00F05082B3F5807F1ED1644AE5
:1050EC00D36C03F04053126812F0040F2DD063BB45
:1050FC005F4B1B68C3F3C1035F48D8409CE77BB18F
:10510C00402B09D15A4B186810F0006094D004A8B9
:10511C00FFF756FC04988FE700208DE700208BE703
:10512C00534B186810F0007086D007A8FFF748FEA4
:10513C00089881E74E4B186810F000503FF47CAF94
:10514C0001A8FFF73DFD019876E7494A126812F471
:10515C00807F03D0B3F1805F00F01082444A126864
:10516C0012F4003F00F00C82B3F1005F00F00A82F1
:10517C00002061E73E4B1B6D03F46063B3F5806F59
:10518C0035D016D9B3F5C06F00F0FE81B3F5006FC2
:10519C0020D1374AD36C03F04053126812F0040F3D
:1051AC0030D07BBB324B1B68C3F3C1033248D840B1
:1051BC0042E78BB1B3F5007F0AD12D4B186810F084
:1051CC0000603FF439AF04A8FFF7FAFB049833E70B
:1051DC00002031E700202FE7254B186810F00070F5
:1051EC003FF42AAF07A8FFF7EBFD089824E7204B04
:1051FC00186810F000503FF41FAF01A8FFF7E0FC57
:10520C00019819E71A4A126812F4807F03D0B3F19F
:10521C00805F00F0BB81164A126812F4003F00F068
:10522C00B781B3F1005F00F0B581002004E7104BAB
:10523C001B6D03F4E043B3F5005F3DD01ED9B3F50D
:10524C00405F00F0A981B3F5804F28D1084AD36C98
:10525C0003F04053126812F0040F38D0002B36D1F3
:10526C00034B1B68C3F3C1030348D840E4E600BFFB
:10527C00004402580080BB000090D0038BB1B3F502
:10528C00805F0AD19F4B186810F000603FF4D4AED9
:10529C0004A8FFF795FB0498CEE60020CCE600208E
:1052AC00CAE6984B186810F000703FF4C5AE07A81A
:1052BC00FFF786FD0898BFE6924B186810F0005077
:1052CC003FF4BAAE01A8FFF77BFC0198B4E68D4A17
:1052DC00126812F4807F03D0B3F1805F00F05E811E
:1052EC00884A126812F4003F00F05A81B3F1005F53
:1052FC0000F0588100209FE6824B1B6D03F4E023E5
:10530C00B3F5403F32D00BD8B3F5803F18D0B3F58E
:10531C00003F20D013B9FEF7FDFC8DE600208BE694
:10532C00B3F5802F2ED0B3F5A02F07D1754B18688D
:10533C0010F400303FF480AE73487DE600207BE62D
:10534C00704B186810F000603FF476AE04A8FFF7BD
:10535C0037FB059870E66B4B186810F000503FF463
:10536C006BAE01A8FFF72CFC029865E6654B18683C
:10537C0010F004003FF460AE1B68C3F3C103634834
:10538C00D84059E65F4B186810F480703FF454AE67
:10539C005F4851E65B4B9B6D03F44033B3F5803FA4
:1053AC0010D0B3F5003F18D0002B40F0FD80554BCA
:1053BC00186810F000603FF43FAE04A8FFF700FB44
:1053CC00049839E64F4B186810F000503FF434AE97
:1053DC0001A8FFF7F5FB03982EE64A4AD36C03F0BD
:1053EC004053126812F0040F07D033B9454B1B68B9
:1053FC00C3F3C1034548D8401EE6424A126812F472
:10540C00807F03D0B3F1805F00F0D0803D4A1268FA
:10541C0012F4003F00F0CC80B3F1005F00F0CA80C2
:10542C00002009E6374BDB6C13F4803302D063B9F0
:10543C00002001E6334B186810F000703FF4FCAD0F
:10544C0007A8FFF7BDFC0898F6E52E4B186810F07E
:10545C0000603FF4F1AD04A8FFF7B2FA0698EBE553
:10546C00284B9B6D03F0E043B3F1405F36D00BD873
:10547C00B3F1805F1CD0B3F1005F24D013B9FFF7F8
:10548C008DFAD9E50020D7E5B3F1A04F32D0B3F1B6
:10549C00C04F00F09180B3F1804F07D1194B1868C1
:1054AC0010F480703FF4C8AD1948C5E50020C3E581
:1054BC00144B186810F000603FF4BEAD04A8FFF761
:1054CC007FFA0598B8E50F4B186810F000503FF4C0
:1054DC00B3AD01A8FFF774FB0298ADE5094B186852
:1054EC0010F004003FF4A8AD1B68C3F3C1030748D8
:1054FC00D840A1E5034B186810F400303FF49CAD84
:10550C00014899E50044025800366E010090D00322
:10551C0000093D002A4B1B6D03F04053B3F1805F33
:10552C000CD0B3F1005F14D0002B47D1244B18687A
:10553C0010F400303FF480AD22487DE5204B186814
:10554C0010F000703FF478AD07A8FFF739FC08980D
:10555C0072E51B4B186810F000603FF46DAD04A8A9
:10556C00FFF72EFA059867E5002065E5164863E518
:10557C00002061E513485FE514485DE512485BE5E2
:10558C00002059E50F4857E5104855E50E4853E5FE
:10559C00002051E50B484FE50C484DE50A484BE51A
:1055AC00002049E5074847E5002045E5064843E566
:1055BC00002041E503483FE504483DE500203BE57C
:1055CC000044025800366E0100093D000080BB000B
:1055DC00F0B4026A036A23F001030362466884692B
:1055EC001E4B23400D681D4322F002028B681343AF
:1055FC001B4A1C4CA04218BF90420CBF0122002237
:10560C000CD004F58044A04214BF00240124164F92
:10561C00B84203D014B9154CA04205D123F00803AD
:10562C00CC68234323F004035AB9114A904214BFA7
:10563C00002201220C4CA04203D012B90B4A90421A
:10564C0005D126F440764A6932438E69164346608A
:10565C0085614A6842630362F0BC70478CFFFEFFB1
:10566C00000001400004014000400140004801409E
:10567C000044014070B4036A026A22F48072026230
:10568C004568C4691A4A22400E68164323F4007315
:10569C008A6843EA0223174A174CA04218BF90426B
:1056AC000CBF0122002206D123F40063CC6843EA2C
:1056BC00042323F480635AB9104A904214BF002289
:1056CC0001220F4CA04203D012B90E4A904207D1CE
:1056DC0025F440524C6942EA04128C6942EA0415E2
:1056EC004560C6614A68C263036270BC704700BF04
:1056FC008CFFFEFF0000014000040140004401400B
:10570C00004001400048014070B4036A026A22F470
:10571C00805202624468C569144A2A400D6842EA04
:10572C00052223F400538D6843EA0533104E114DC6
:10573C00A84218BFB0420DD005F58045A84214BF51
:10574C000025012506F58046B04203D015B90A4D57
:10575C00A84204D124F480444D6944EA8514446081
:10576C00C2614A680264036270BC7047FF8CFFFE22
:10577C0000000140000401400048014070B4036A7D
:10578C00026A22F4803202624268456D144E2E4049
:10579C000D682E4323F400338C6843EA0443114D07
:1057AC00114CA04218BFA8420DD004F58044A04271
:1057BC0014BF0024012405F58045A84203D014B978
:1057CC000A4CA04204D122F480324C6942EA0422F1
:1057DC00426046654A688265036270BC704700BFD0
:1057EC008FFFFEFF00000140000401400048014013
:1057FC0070B4036A026A22F4801202624468456D36
:10580C00144A2A400D6842EA052223F400138D68DD
:10581C0043EA0553104E114DA84218BFB0420DD0AB
:10582C0005F58045A84214BF0025012506F58046E4
:10583C00B04203D015B90A4DA84204D124F48024F7
:10584C004D6944EA8524446042654A68C265036236
:10585C0070BC7047FF8FFFFE000001400004014048
:10586C000048014010B4036A046A24F00104046285
:10587C00846924F0F00C4CEA021223F00A030B4367
:10588C00826103625DF8044B704730B4056A046AA8
:10589C0024F010040462846924F4407C4CEA022C49
:1058AC002CF4704C1B039BB243EA0C0325F0A005AF
:1058BC00090101F0A00129438361016230BC7047EA
:1058CC0010B4036A046A24F010040462846924F49A
:1058DC00704C4CEA023223F0A00343EA01138261BC
:1058EC0003625DF8044B704730B4056A046A24F413
:1058FC0080740462C46924F0030C4CEA020C2CF092
:10590C00F00C1B01DBB243EA0C0325F42065090201
:10591C0001F420612943C361016230BC704730B48B
:10592C00056A046A24F480540462C46924F4407C3B
:10593C004CEA022C2CF4704C1B039BB243EA0C0374
:10594C0025F42045090301F420412943C361016278
:10595C0030BC70478268034B13400B4343F0070382
:10596C00836070478FFFCFFF70B40368394A904251
:10597C0014BF00220122B0F1804F14BF144642F034
:10598C000104ACB9344DA84214BF00250125334E97
:10599C00B0420DD065B905F1804505F58235A842B8
:1059AC0014BF0025012506F50066B04200D01DB1DC
:1059BC0023F070034D682B4314BB274CA04214BF3B
:1059CC0000240124254DA8421AD0CCB904F18044FE
:1059DC0004F58234A04214BF0024012405F50065AF
:1059EC00A8420DD064B91E4CA04214BF002401245F
:1059FC0005F59A35A84203D014B91A4CA04203D12C
:105A0C0023F44073CC68234323F080034C69234375
:105A1C008C68C4620C688462134CA04208BF42F0CC
:105A2C00010262B90E4A904214BF0022012204F511
:105A3C007054A04203D012B90A4A904201D10A69AB
:105A4C000263026842F004020260012242610360B8
:105A5C0070BC70470000014000080040000400408A
:105A6C0000440140004801400004014060B310B5FF
:105A7C00044690F83D3013B3022384F83D302146A0
:105A8C0051F8040BFFF770FF012384F8483084F8B9
:105A9C003E3084F83F3084F8403084F8413084F84C
:105AAC00423084F8433084F8443084F8453084F82C
:105ABC00463084F8473084F83D30002010BD80F823
:105ACC003C30FDF751FAD7E70120704760B310B5B1
:105ADC00044690F83D3013B3022384F83D30214640
:105AEC0051F8040BFFF740FF012384F8483084F889
:105AFC003E3084F83F3084F8403084F8413084F8EC
:105B0C00423084F8433084F8443084F8453084F8CB
:105B1C00463084F8473084F83D30002010BD80F8C2
:105B2C003C30FDF74DFAD7E70120704760B310B554
:105B3C00044690F83D3013B3022384F83D302146DF
:105B4C0051F8040BFFF710FF012384F8483084F858
:105B5C003E3084F83F3084F8403084F8413084F88B
:105B6C00423084F8433084F8443084F8453084F86B
:105B7C00463084F8473084F83D30002010BD80F862
:105B8C003C30FDF749FAD7E70120704770B4036A3F
:105B9C00026A22F010020262456884691A4E26409D
:105BAC000C6846EA042623F020038A6843EA0213B1
:105BBC00164A174CA04218BF90420CBF012200227B
:105BCC0006D123F08003CC6843EA041323F040038E
:105BDC005AB9104A904214BF002201220E4CA04226
:105BEC0003D012B90D4A904207D125F4406C4A6992
:105BFC004CEA820C8A694CEA8205456086614A68E7
:105C0C008263036270BC7047FF8CFFFE0000014092
:105C1C0000040140004401400040014000480140A4
:105C2C0038B590F83C30012B00F0958004460D46B9
:105C3C00012380F83C30142A00F28880DFE802F05F
:105C4C000B8686861F86868634868686488686865A
:105C5C005D86868671000068FFF7BAFC226893693E
:105C6C0043F0080393612268936923F00403936162
:105C7C002268936929690B439361002067E00068EF
:105C8C00FFF784FF2268936943F4006393612268F1
:105C9C00936923F48063936122689369296943EAC9
:105CAC0001239361002052E00068FFF7E3FC2268B7
:105CBC00D36943F00803D3612268D36923F004034A
:105CCC00D3612268D36929690B43D36100203EE07C
:105CDC000068FFF719FD2268D36943F40063D361B0
:105CEC002268D36923F48063D3612268D36929695C
:105CFC0043EA0123D361002029E00068FFF73EFD51
:105D0C002268536D43F0080353652268536D23F0EA
:105D1C00040353652268536D29690B4353650020B6
:105D2C0015E00068FFF764FD2268536D43F40063CF
:105D3C0053652268536D23F4806353652268536D59
:105D4C00296943EA01235365002000E00120002368
:105D5C0084F83C3038BD0220FCE7000070B4944657
:105D6C00066A046A24F00104046284691D4DB0F1D2
:105D7C00804F18BFA84223D01B4A904214BF002268
:105D8C000122A5F57C45A8421AD0CAB902F180427D
:105D9C0002F58232904214BF0022012205F5006503
:105DAC00A8420DD062B9114A904214BF00220122C0
:105DBC0005F54065A84203D012B944F0010203E096
:105DCC0024F0030242EA0C0222F0F0021B01DBB2C7
:105DDC00134326F00A0201F00A01114383610162A8
:105DEC0070BC7047000001400008004000400140BA
:105DFC0038B590F83C30012B5ED004460D4601239B
:105E0C0080F83C300C2A52D8DFE802F0075151518F
:105E1C00195151512C5151513E00CB684A680968B7
:105E2C000068FFF79BFF2268936923F00C039361D2
:105E3C0022689369A9680B439361002038E0CB6812
:105E4C004A6809680068FFF720FD2268936923F40B
:105E5C004063936122689369A96843EA01239361C3
:105E6C00002025E0CB684A6809680068FFF73CFD14
:105E7C002268D36923F00C03D3612268D369A96823
:105E8C000B43D361002013E0CB684A6809680068B3
:105E9C00FFF745FD2268D36923F44063D361226880
:105EAC00D369A96843EA0123D361002000E00120F3
:105EBC00002384F83C3038BD0220FCE710B4846821
:105ECC0024F47F4C42EA03220A4342EA0C02826029
:105EDC005DF8044B7047000090F83C30012B00F04B
:105EEC008F8010B50446012380F83C30022380F8E3
:105EFC003D3002689068434B034093600B68702BF5
:105F0C0055D031D8502B6CD01FD8402B0AD1CA6831
:105F1C0049682068FFF7A6FC40212068FFF71AFDAE
:105F2C00002029E068D8202B03D00AD80BB1102B05
:105F3C0005D119462068FFF70DFD00201CE001205B
:105F4C001AE0302BF5D0012016E0602B0AD1CA687C
:105F5C0049682068FFF7B4FC60212068FFF7FAFC61
:105F6C00002009E0012007E0B3F5005F2CD00AD82F
:105F7C00B3F5805F42D10020012384F83D3000232B
:105F8C0084F83C3010BD204A9342D2D007D8B3F5E8
:105F9C00801FCED0B3F1101FCBD00120ECE71B4AF1
:105FAC009342C6D010329342C3D00120E4E7CB68B1
:105FBC004A6889682068FFF781FF2268936843F07C
:105FCC00770393600020D7E7CB684A68896820681C
:105FDC00FFF774FF2268936843F4804393600020BA
:105FEC00CAE7CA6849682068FFF73CFC5021206862
:105FFC00FFF7B0FC0020BFE70120BDE70120BBE7A5
:10600C00022070478800CEFF2000100030001000E6
:10601C0090F83C20012A45D070B40346012280F848
:10602C003C20022280F83D200268506894681E4E85
:10603C001E4DAA4218BFB24203D120F470004D6825
:10604C00284320F070000D68284350601A681648E9
:10605C00B2F1804F18BF824217D0A0F57C4082422B
:10606C0013D000F5806082420FD000F58060824230
:10607C000BD000F57840824207D0A0F56C408242EC
:10608C0003D000F59430824204D124F08004896856
:10609C0021439160012283F83D20002083F83C00CD
:1060AC0070BC7047022070470000014000040140A2
:1060BC0090F83C30012B44D030B40246012380F8D8
:1060CC003C30CB6823F440738868034323F480632B
:1060DC004868034323F400630868034323F48053A4
:1060EC000869034323F400534869034323F48043B2
:1060FC00086B034323F47023886943EA004323F0BD
:10610C008053C869034310680F4D104CA04218BF50
:10611C00A84210D123F470038C6A43EA045323F091
:10612C0080730C6A234323F000734C6A234323F0DF
:10613C000053C96A0B434364002082F83C0030BC16
:10614C0070470220704700BF00000140000401406E
:10615C00FEE7FEE7FEE7FEE7FEE770477047704795
:10616C0008B5FAF7E9FC08BD08B50248FBF7A8FE2C
:10617C0008BD00BFE802002008B50248FAF74AFD46
:10618C0008BD00BF600300202B4AD2F8883043F4CE
:10619C007003C2F88830294B1B6803F00F03022BE5
:1061AC0006D8264A136823F00F0343F00303136049
:1061BC00234B1A6842F001021A6000221A61196816
:1061CC00204A0A401A601D4B1B6813F00C0F06D0B6
:1061DC001A4A136823F00F0343F003031360184BA0
:1061EC0000229A61DA611A62174999621749D962D9
:1061FC00174919635A639963DA6319645A64196805
:10620C0021F4802119601A66D3F8343113F4805FBD
:10621C0010D10B4BD3F8342142F48052C3F8342103
:10622C000C4A43F2D2011160D3F8342122F480528B
:10623C00C3F83421704700BF00ED00E0002000528D
:10624C00004402587FEDF6EA000202020000FF0152
:10625C008002010100400052054AD36843F002035A
:10626C00D360034B5B6813F4005FFAD0704700BF38
:10627C0000480258DFF838D0FFF7EEFFFFF784FF35
:10628C000C480D490D4A002302E0D458C450043385
:10629C00C4188C42F9D30A4A0A4C002301E013605B
:1062AC000432A242FBD300F019F8FAF791FB7047C5
:1062BC00000002200000002010000020D063000825
:1062CC0010000020CC030020FEE70244034693425A
:1062DC0000D1704703F8011BF9E7000070B50D4BB6
:1062EC000D4D5B1B9C100026A64209D100F028F82E
:1062FC000A4D0B4B5B1B9C100026A64205D170BDB2
:10630C0055F8043B98470136EEE755F8043B98479F
:10631C000136F2E7C8630008C8630008C8630008C8
:10632C00CC6300080A44914200F1FF3300D170475E
:10633C0010B511F8014B03F8014F9142F9D110BD82
:10634C00F8B500BFF8BC08BC9E467047F8B500BF56
:08635C00F8BC08BC9E46704726
:106364000000000000000000000000000000000029
:106374000000000001000000020000000300000013
:106384000400000000000000050000000000000000
:1063940000000000000000000600000000000000F3
:1063A40000000000000000000700000000061016B6
:1063B4000006101600000000010203040102030499
:0463C40006070809B7
:0463C800D1020008F6
:0463CC00AD02000816
:1063D00001000000100000000090D0030090D003E6
:04000005080062810C
:00000001FF
